:020000040000FA
:10000000BDEF0AF01200FFFFFFFFFFFFFFFFFFFF42
:10080000BDEF0AF01200FFFFFFFFFFFFFFFFFFFF3A
:10081000FFFFFFFFFFFFFFFFFFFFFFFFFFFFFFFFE8
:10082000FFFFFFFFFFFFFFFFFFFF01009A15000022
:10083000820000000300000004011051600BE84238
:10084000E842E842E842E842000901E055D011518F
:10085000070A51E00B0A4FE0070A40E0010A2CE0CA
:100860000B0A28E0020A26E0030A22E0080A12E046
:10087000010A0EE00F0A0AE0030A01E03CD0000181
:10088000010E746F0001040E7B6F36D036D834D061
:1008900090D832D00001010E746F00017D0E756F8B
:1008A000000E766F00017C930001010E796F24D059
:1008B000A8D822D0F6D820D00001010E746F040110
:1008C00014510001756F766B7E0E7527000E76232E
:1008D00000017C930001010E796F0ED00001010E22
:1008E000746F04011451EA6A7E0FE96E000EEA2269
:1008F00012C4EFFF01D000D01200800E0401105D81
:1009000057E11351030A34E0010A10E0030A01E041
:100910004DD00001010E746F0001CE0E756F130EE5
:10092000766F120E0001796F7A6B40D00001010ED4
:10093000746F04011251F66EF76AD890F636F736E6
:100940009A0EF626140EF7220900F5CF75F00A006C
:10095000F5CF76F0020E0001F76A7525F66E765136
:10096000F7220900F5CF79F00A00F5CF7AF01ED012
:100970000001010E746F04011251F66EF76AD890EF
:10098000F636F7369E0EF626140EF7220900F5CF3E
:1009900075F00A00F5CF76F075C0F6FF76C0F7FF68
:1009A0000800F5500001796F7A6B00D000017C835C
:1009B00012000001010E746F0F0EE66E710EE66EEE
:1009C0000F0EE66ED2EC09F0E552E552E552010E4B
:1009D000E66E7E0EE66E000EE66ED2EC09F0E55293
:1009E000E552E55212C47DF00401125104E1000108
:1009F000050E7B6F05D00001060E7B6FA1EC07F0A2
:100A000012000401186B196B040110511F0B020A2C
:100A100016E0030A10E0010A01E035D00001010EE2
:100A2000746F80A402D00401188100017CA102D05F
:100A30000401188328D00001010E746F24D0000136
:100A4000010E746F040114510F0B080DF350036A6B
:100A5000000F026E040E03221451800B01E0010E00
:100A6000040DF35000010224776F000E0320786F0D
:100A700077C0E9FF78C0EAFFEF50040B03E0040100
:100A8000010E186F00D0000174050AE10001180E74
:100A9000756F040E766F00017C930001020E796F72
:100AA00012000401120510E110511F0B00090CE1A6
:100AB0000001010E746F030E0401115D03E10001DA
:100AC0007C8102D000017C91040112513AE1105165
:100AD0001F0B020836E114510F0B000932E0000130
:100AE000010E746F040114510F0B080DF350036ACB
:100AF000000F026E040E03221451800B01E0010E60
:100B0000040DF35000010224776F000E0320786F6C
:100B1000030E0401115D07E1840E77C0E9FF78C080
:100B2000EAFFEF6E0ED014AF06D077C0E9FF78C0B1
:100B3000EAFFEF6A06D0880E77C0E9FF78C0EAFFC7
:100B4000EF6E12006C5002E0000E01D0010E0009A1
:100B50000BE0040100513C0BE842E8420D0802E1C1
:100B60000CD801D040D808D06C5002E0000E01D063
:100B7000010E040901E047D81200D9CFE6FFE1CF0A
:100B8000D9FFE6520001736B746B796B7A6B1CECC6
:100B900004F0DF6ADF50026E036A010E025C000E91
:100BA00003581BE20001745101E017D0F76ADF34EB
:100BB000FE0BF736F66EA40EF626140EF722090089
:100BC000F5CF02F00800F5CF03F004D003C0FAFF20
:100BD0000250F96EFBDFDF2ADDD7DDD8E552E552A2
:100BE000E7CFD9FF1200020E0001735D0AE196D82B
:100BF000040100BD03D0C80E006F02D0880E006F44
:100C000001D00FD91200040E00017B5D0AE112C46D
:100C10006EFF6E50000803E2050E7B6F02D0030EDC
:100C20007B6F000173050AE10BD8040104BD03D0FA
:100C3000C80E046F02D0880E046F01D0F2D81200E3
:100C4000D9CFE6FFE1CFD9FF020EE1260001080E61
:100C5000795D000E7A5905E279C0DEFF7AC0DDFFCA
:100C600003D0080EDE6EDD6A040104930491010EC8
:100C7000DB500413DFCF05F4000EDB500001795F79
:100C8000010EDB507A5B180E776F040E786F00014F
:100C90007CA31ED0D9CFE9FFDACFEAFFEE50ED10EA
:100CA00016E075C0F6FF76C0F7FF0800F55077C074
:100CB000E9FF78C0EAFFEF6E0001772B000E782382
:100CC000752B7623DF06010E01E2DB06E3D71CD08D
:100CD000D9CFE9FFDACFEAFFEE50ED1015E075C08D
:100CE000E9FF76C0EAFFEF5077C0E9FF78C0EAFF7E
:100CF000EF6E0001772B000E7823752B7623DF062D
:100D0000010E01E2DB06E4D7020EE15C02E2E16AD9
:100D1000E552E16EE552E7CFD9FF1200D9CFE6FFE9
:100D2000E1CFD9FF020EE126030E04010015E76EA4
:100D3000010EE7CFDBFF01C4DFFFDE5000017927A2
:100D4000DD507A23180E756F040E766FD9CFE9FF48
:100D5000DACFEAFFEE50ED1014E075C0E9FF76C07F
:100D6000EAFFEF5077C0E9FF78C0EAFFEF6E772B1C
:100D7000000E7823752B7623DF06010E01E2DB06D9
:100D8000E5D7020EE15C02E2E16AE552E16EE5526E
:100D9000E7CFD9FF1200000174510CE10401080EE5
:100DA000016F100E026F040E036F840E006F0401BA
:100DB000046F35D0040110AF22D000017951040135
:100DC000165D00017A510401175904E216C479F046
:100DD00017C47AF035DF0001010E736F0401080EAD
:100DE000016F100E026F040E036F800E006F04017E
:100DF000180E066F040E076FC80E046F10D00001A6
:100E0000020E736F0401056BC80E046F0401080E17
:100E1000016F180E026F040E036FC80E006F6D98FD
:100E200012000001736B0401080E016F100E026FB7
:100E3000040E036F880E006F0401046B120004019E
:100E400010511F0B010801E079D0145101E076D058
:100E5000060E115D2EE11351230A28E0010A13E06A
:100E6000030A01E024D00001020E746F00017D0529
:100E700005E10001F20E756F130E766F090E000189
:100E8000796F7A6B14D00001020E746F00017D053A
:100E900005E10001680E756F140E766F00017D0587
:100EA00004E1320E0001796F7A6B01D000D00001AD
:100EB0007C8304011051600BE842E842E842E842BA
:100EC000E842010801E03AD011510B0A31E0080A6A
:100ED00021E0090A19E0080A09E00B0A05E0080AFE
:100EE00001E02CD02CD82AD02BD828D00001020E1B
:100EF000746F00017F0E756F000E766F00017C939A
:100F00000001010E796F1AD00001020E746F13C434
:100F10007FF014D00001020E746F0001800E756F17
:100F2000000E766F00017C930001010E796F06D0F0
:100F30000001020E746F12C480F000D01200120083
:100F400012000001816B1E0E716E0401030E096F09
:100F5000200E0A6F040E0B6F880E086F0401230E1B
:100F60000E6F040E0F6F400E0C6F1200D9CFE6FF0C
:100F7000E1CFD9FFE652FC0EDB50030805E2030E79
:100F8000F36EFC0EF3CFDBFFDF6AFC0EDB50DF5CA1
:100F900019E2DF50E76EFD0EDBCFE9FFFE0EDBCF7F
:100FA000EAFFE750E926000EEA22EF50E66EDF5036
:100FB000EA6A230FE96E040EEA22E552E750EF6E6B
:100FC000DF2AE3D7FC0EDBCF0DF4400E04010C1733
:100FD0000C7D880E0C13E552E552E7CFD9FF1200C5
:100FE000D9CFE6FFE1CFD9FF0001816B040108BF33
:100FF00031D0FC0EDBCF02F00951D880025403E25D
:10100000FC0E09C4DBFF0001816BFC0EDB50815D2F
:1010100019E28151EA6A200FE96E040EEA22EF50CC
:10102000E66E8151E76EFD0EDBCFE9FFFE0EDBCFF2
:10103000EAFFE750E926000EEA22E552E750EF6E9C
:10104000812BE3D70401030E096F400E0817087DBA
:10105000880E08130001815100D0E552E7CFD9FF77
:101060001200F00E8C1695169388938A938C938EAB
:101070008150200B01E0010E00016A6F8150100BBE
:1010800001E0010E6B6F8150800B01E0010E6C6F6F
:101090008150400B01E0010E6D6F706B716B726BD4
:1010A000736B010E6E6F120039D8060E00017B5D66
:1010B00003E36D50020B01E001D001D812000001E2
:1010C0006E0516E1706B81BA02D0726906D081B8E4
:1010D00003D0010E726F01D0726B81BE03D0010E7E
:1010E000716F05D081BC02D0716901D0716B05D0E0
:1010F000726B72C071F072C070F004010CBF0DD041
:10110000030EE66E700EE66E000EE66EB6EC07F0AD
:10111000E552E552E55200016F2B120000018351A8
:10112000841104E1100E836F270E846F8307000E75
:10113000845B6DA20BD08351841107E18C708C50BD
:10114000010B02E08C8201D08C922FD000017B51E8
:1011500003E18C908C9229D07B0503E18C808C82FA
:1011600024D0020E7B5D03E18C808C921ED0030E96
:101170007B5D03E18C908C8218D0050E7B5D07E1CE
:1011800000018351841102E18C708C920ED0060E06
:101190007B5D0BE100018351841107E18C708C5061
:1011A000010B02E08C9201D08C8212008150200B46
:1011B00001E0010E00016A5D09E08150200B01E0B1
:1011C000010E6A6F81BA02D0010E02D0000E00D06B
:1011D00012008150100B01E0010E00016B5D09E06F
:1011E0008150100B01E0010E6B6F81B802D0010E2F
:1011F00002D0000E00D012008150800B01E0010EE1
:1012000000016C5D09E08150800B01E0010E6C6F04
:1012100081BE02D0010E02D0000E00D0120081501B
:10122000400B01E0010E00016D5D09E08150400BB3
:1012300001E0010E6D6F81BC02D0010E02D0000EE4
:1012400000D0120080A203D06DA60FD802D06DB6D8
:1012500013D800017B0508E16DBA06D0686A696A97
:1012600069806988020E7B6F12006D6A696A6D86FB
:101270000001010E7B6F12006D6A696A00017B6BD1
:1012800012003CEF09F000017B5101E13AD06850B7
:10129000040B04E06950040B01E041D86DB231D079
:1012A0006850010B04E06950010B01E059D8685007
:1012B000100B04E06950100B01E024D86850400B7B
:1012C00004E06950400B01E040D86850200B04E076
:1012D0006950200B01E03BD86850020B04E06950D4
:1012E000020B01E03BD8030E00017B5D01E209D057
:1012F0006850080B06E06950080B03E0A2EC05F00B
:1013000068961200698468986D82A19AF290A08A0A
:10131000F2860300F2B007D8A09AF29612006D92FE
:1013200069946894120000017CA10ED0F8DF6D84EE
:101330000001080E856F070E866F8507000E865B1D
:1013400085518611FAE16D941200689C120070A01C
:1013500003D011EC07F07090689A120068921200A6
:101360006A6A686A9F0E6B6E7B0E696E6E6A0F0EFC
:10137000E66E710EE66E0F0EE66E14D8E552E5527B
:10138000E552160E706E68A602D06896FCD76D986E
:1013900011EC07F000017C9100017D6B0001030E50
:1013A0007B6F1200D9CFE6FFE1CFD9FFFD0EDBCF77
:1013B000E9FFFE0EDBCFEAFFFC0EDB5004E0EE6A35
:1013C000FC0EDB06F9D7E552E7CFD9FF1200120178
:1013D000000200000008D804000001000102000122
:1013E00009022200010100A03209040000010301EA
:1013F00002000921010100012232000705810303D7
:10140000000A0403090434034D00690063007200FC
:101410006F006300680069007000200054006500E0
:10142000630068006E006F006C006F006700790059
:10143000200049006E0063002E002E034D006F0057
:10144000750073006500200049006E0020006100F7
:10145000200043006900720063006C0065002000FA
:10146000440065006D006F0005010902A10109013A
:10147000A10005091901290315002501950375012E
:101480008102950175058101050109300931158138
:10149000257F750895028106C0C0E013E013021491
:1014A00006143A143E0E2A0EF66E080EF76E000E63
:1014B000F86E00010900F550656F0900F550666F80
:1014C00003E1656701D03DD00900F550606F090068
:1014D000F550616F0900F550626F09000900F55081
:1014E000E96E0900F550EA6E090009000900F5509F
:1014F000636F0900F550646F09000900F6CF67F0CB
:10150000F7CF68F0F8CF69F060C0F6FF61C0F7FF71
:1015100062C0F8FF0001635302E1645307E0090071
:10152000F550EE6E6307F8E26407F9D767C0F6FF7F
:1015300068C0F7FF69C0F8FF00016507000E665B31
:10154000BFD7120005D812D854EC08F0FCD712000F
:101550000F0EC11292829284140E6F6E00017B6B8B
:1015600000017C6B00017D6B31EF08F022EC09F08B
:101570006FBE02D043EC09F0120013EE00F023EE30
:1015800000F0F86A019C53EC0AF0A2EC0AF0FDD7D7
:101590001200FCFCFC0004040400000000FFFFFF3C
:0200000400F00A
:10000000FFFFFFFFFFFFFFFFFFFFFFFFFFFFFFFF00
:10001000FFFFFFFFFFFFFFFFFFFFFFFFFFFFFFFFF0
:10002000FFFFFFFFFFFFFFFFFFFFFFFFFFFFFFFFE0
:10003000FFFFFFFFFFFFFFFFFFFFFFFFFFFFFFFFD0
:10004000FFFFFFFFFFFFFFFFFFFFFFFFFFFFFFFFC0
:10005000FFFFFFFFFFFFFFFFFFFFFFFFFFFFFFFFB0
:10006000FFFFFFFFFFFFFFFFFFFFFFFFFFFFFFFFA0
:10007000FFFFFFFFFFFFFFFFFFFFFFFFFFFFFFFF90
:10008000FFFFFFFFFFFFFFFFFFFFFFFFFFFFFFFF80
:10009000FFFFFFFFFFFFFFFFFFFFFFFFFFFFFFFF70
:1000A000FFFFFFFFFFFFFFFFFFFFFFFFFFFFFFFF60
:1000B000FFFFFFFFFFFFFFFFFFFFFFFFFFFFFFFF50
:1000C000FFFFFFFFFFFFFFFFFFFFFFFFFFFFFFFF40
:1000D000FFFFFFFFFFFFFFFFFFFFFFFFFFFFFFFF30
:1000E000FFFFFFFFFFFFFFFFFFFFFFFFFFFFFFFF20
:1000F000FFFFFFFFFFFFFFFFFFFFFFFFFFFFFFFF10
:020000040030CA
:0E000000240E3F1E008181000FC00FA00F4094
:020000040020DA
:08000000FFFFFFFFFFFFFFFF00
:00000001FF
